:020000040000FA
:1000000083168601EF308500C13081008312A5017F
:10001000A701A901A801C830AB00F630AE00A320AB
:10002000051D1B280130AC001430A9002814A814A9
:100030004B20F8203D28AC014B208730FE20640087
:100040001F288207C034F934A434B0349934923470
:100050008234F8348034903482073134B734313408
:10006000743431347E34313488343134943431341E
:10007000AB343134B13431346034A320E820AA0BDE
:100080003D2864001130AA00C120AB0B3D28283068
:10009000AB00A9203D2803102C0DA6002C20A100A8
:1000A000260A2C20A0006430A4000310A00DA10D8E
:1000B00020146820C4307520003075202008752079
:1000C0002108752024087520003075209020080034
:1000D0000C3083168500831285140000051400007F
:1000E00085100000051000000800A3000C308316E6
:1000F000850083120830A200A30D8514031C85100F
:1001000000000514000005100000A20B7C280E3032
:1001100083168500831205140000051000000800F6
:100120000C30831685008312851000000514000032
:10013000851400000F308316850083120800FE30FE
:10014000AE00AD0108000B1DA328B93081000B11D2
:100150000800A9080319B6288519BF284B30A90043
:10016000A81CB528D230AE00A8100800281CBB2857
:10017000F2204B20F820A8141430A900B528A903B8
:10018000B528A708031DD0280519CF289F20A50151
:100190000A30A7002818E228F2204B20F820080097
:1001A0000519E0280A30A700A50A64302502031DBE
:1001B000CF282814A8141430A90086139F20CF2814
:1001C000A703CF280F30A900A81028108617CF2822
:1001D000AE080319F1280130AD070318AE0A10303C
:1001E0008506080007302C020318AC01AC0A080091
:1001F0002C082120FE2028188613080086000800FD
:02400E00FD3F74
:00000001FF
